:020000020000FC
:100000000C94050A6DC20000000000000000000012
:1000100000000000000000000000000000000000E0
:100020000000000033C00000000000005DC10000BF
:1000300000000000000000000000000000000000C0
:1000400059C1000000000000000000000000000096
:100050000000000002030406080C10182030406065
:10006000800002030406080C101820304080FF00B6
:100070000406080C10182030406080A0C0000D0D50
:100080000405060D050D0602030302004FB662FDCE
:1000900020C070FF1BC165FDFBC00994C0913701F2
:1000A000C395C0933701C5E0C519B8F3D0913701A6
:1000B000CD1B98F3C8E7089483FDC795C093B200A1
:1000C000C52DCC2329F4C0E083FDC0E8C093B20065
:1000D00009C171FF03C02B982C982D98C52D089449
:1000E00083FDC795C093B200C09339016B7FC52DC6
:1000F000CF3F09F441C0C0913801C395C093380186
:1001000070FF35C02B982C982D984FBE18957860AD
:10011000C0914001CC2391F0C0913801CA95D09193
:100120004001CD1B58F0777FC0913801D0913F013D
:10013000CD1B08F41CC02092380119C02B982C98B4
:100140002D98C1E0CA95F1F7C0911501CA95C2FD7D
:1001500009C0C1FD05C095FF299A95FD2A9A0EC0D8
:10016000289A0CC095FF2A9A95FD299A07C02B98CA
:100170002C982D984FBE1895209239014FBE189596
:10018000A5C0552021F095FF2B9A95FD2D9A2C980E
:100190009DC0552009F02C9A95FF2D9895FD2B9820
:1001A00095C0552021F095FF2D9A95FD2B9A95FF2E
:1001B0002B9895FD2D988AC095FF2A9895FD299832
:1001C00095FF299895FD2A98C1E0CA95F1F7552029
:1001D00021F095FF2B9A95FD2D9A2C9877C095FFCD
:1001E0002A9895FD29982898C1E0CA95F1F75520DD
:1001F00021F095FF2B9A95FD2D9A2C9867C0289891
:1002000095FF2A9895FD2998C1E0CA95F1F75520E8
:1002100009F02C9A95FF2D9895FD2B9857C028989A
:1002200095FF299895FD2A98C1E0CA95F1F75520C8
:1002300009F02C9A95FF2D9895FD2B9847C095FFB6
:10024000299895FD2A982898C1E0CA95F1F755207C
:1002500021F095FF2D9A95FD2B9A95FF2B9895FDF2
:100260002D9834C095FF299895FD2A9895FF2A98D6
:1002700095FD2998C1E0CA95F1F7552021F095FF29
:100280002D9A95FD2B9A95FF2B9895FD2D981EC0C4
:1002900082FF1CC0C0911501C2FD0BC0C1FD11C081
:1002A00095FF2A9895FD299895FF299895FD2A98FC
:1002B0000DC0C1FDF5CF95FF2A9895FD2998289886
:1002C00005C0289895FF299895FD2A98C52DC095B9
:1002D000089483FDC795C093B200C0933901209262
:1002E000370164604FBE18954FB6C2E0C6BB6E7F43
:1002F0004FBE18953FB68F7EADB3A170A21180613D
:10030000A0E0ADBBA0916E00AE7FA0936E0078948C
:10031000A0910601AA2349F0A92FAF7159F1A0912C
:100320000601AA95A093060125C040E050E0A9B1BE
:1003300096FDA095A2FD4FEF96FFA3E096FDA2E0EB
:10034000A0936900AA27A160ACBB8D7FA9B196FDDF
:10035000A095A2FD5FEF451741F7A8E161FDA093CD
:100360000601A92FAF7119F0A8E1A09306014093EF
:100370002D018160A0910701AA2331F0A09107010E
:10038000AA95A093070107C0A92FAF7121F0806142
:10039000AA27A160ACBB80FF4BC0A0912D014A2FC2
:1003A0008E7FA92FAF71E1F0A0914E01A430C1F46E
:1003B000403F08F040EFA42FA295AF704A0F509134
:1003C0005001533069F0A695A69550FD01C0A69541
:1003D00052FD03C0A41B4A2F03C04A0F08F44FEF7D
:1003E0004093010171FF08C0A091010150913201B9
:1003F000A51710F05093010140914E01443029F5AA
:10040000A091010140910301A41B70F040916F0184
:10041000A40B50F0A0910301A40FA093030140F49A
:10042000AFEFA093030104C0A0910101A0930301C9
:1004300040910301A09132014A1708F04A2FA09180
:1004400034014A1708F04A2F542EA52DA03408F085
:100450006860A0910001A395A093000161F0F89459
:10046000A0916E00A160A0936E0084FF02C0A1E085
:10047000ADBB3FBE189541E050910601552331F0C8
:10048000A92FAF7119F45A9550930601A0912D012F
:10049000A13018F0209230010DC02092310120923D
:1004A0003A01A0913001AF5FA093300118F0AFEF97
:1004B000A0933001A0913301A65F20F05FEF50932D
:1004C000330102C0A0933301F894A0916E00A160A3
:1004D000A0936E0084FF02C0A1E0ADBB3FBE1895A3
:1004E0003FB640918400509185008F7EADB3A170DE
:1004F000A2118061A0E0ADBBA0916E00AE7FA09381
:100500006E00789481FD28C096FFA2E096FDA3E0DE
:10051000A09369008260A9B196FDA095A2FF05C0D5
:10052000409304015093050136C196FFA3E096FD68
:10053000A2E0A0936900AA27A160ACBB8D7FA92F80
:10054000AF7109F419C140E0A9B196FDA095A2FDD3
:1005500013C140932D0106C196FFA3E096FDA2E0D2
:10056000A09369008D7F61FF6CC096FFA2E096FDAD
:10057000A3E0A0936900AA27A160ACBB826040936E
:10058000280150932901A09026014A19B090270113
:100590005B09BB24A2E0EA2EA22C483CA0E05A074B
:1005A00030F4A0E1BA2EE22CAAE0AA2E27C04836E9
:1005B000A1E05A0730F4A8E0BA2EE22CAFE0AA2E50
:1005C0001DC0403DA2E05A0730F4A4E0BA2EE22C50
:1005D000AEE1AA2E13C0403AA5E05A0730F4A2E0DB
:1005E000BA2EE22CACE3AA2E09C04839A8E05A077B
:1005F00028F4A1E0BA2EE22CA8E7AA2EC42EA091DE
:100600002A01CA1AD52EA0912B01DA0ADD202AF47C
:10061000AFEFC094D094CA1ADA0A20922C01CA14FF
:10062000DE0418F4A1E0A0932C0140932A0150931A
:100630002B014091280150912901409326015093AC
:100640002701A09104014A1BA09105015A0B94FDBA
:100650007CC093FD7AC092FD76C05695479591FD7A
:1006600072C05695479590FD6EC0D52EC42ED69477
:10067000C79461FD0CC0AC2DAC51AD2DA24008F06B
:100680007BC0DD2021F4AC2DA85C08F475C0A0E08F
:10069000EA2E97FD08C0E0906201A0915401A330BA
:1006A00011F4E0906A01AAEFEA0EF22CF21CCE18C7
:1006B000DF084FB74170A0915401A330A9F444233F
:1006C00029F095FD11C0F894906204C095FF0CC00C
:1006D000F8949F7D2B982C982D982A9828982998E3
:1006E00071FD01C060687894442369F0A0915401C1
:1006F000A33031F4AFEFC094D094CA1ADA0A03C021
:1007000040E050E022C0A0915401A33049F4CC0C49
:10071000DD1CA5E0CA1AD20818F4A0E0CA2ED22C1B
:10072000AFEFCA16D20418F04FEF50E00EC0F090B1
:100730004701CF9C412D000C441F50E008F012C02F
:100740004FEF50E00FC05695479594FF07C05523D3
:1007500009F04FEFA42FA6954A0F521D4F3F5205A7
:1007600008F04FEF40932D01816061FF05C0AFE1BC
:10077000A095A923AB299A2FA8E1A0930601A92F40
:10078000AF7119F4AAE0A093060161FD04C0A92F7E
:10079000AF7109F08F7EA6E0A0930701A92FAF717A
:1007A00019F4AAE0A0930701F894A0916E00A1604B
:1007B000A0936E0084FF02C0A1E0ADBB3FBE1895C0
:1007C00011E00AC013E008C01AE006C01EE104C030
:1007D00014E602C018EC00C005E1BB27BA95F1F79A
:1007E0000A95D9F71A95C1F708952AE338E709C0A1
:1007F00020E33CE806C02AE234EB03C025E238ECF3
:1008000000C0652CB1E05B2E12E095FD9F7D95FF49
:100810009062BB272898BA95F1F7552009F02C9AD9
:10082000BA95F1F72C98BA95F1F7289ABA95F1F79D
:10083000552021F095FF2B9A95FD2D9AB0914801F6
:10084000BA95F1F795FF2B9895FD2D98B7E8BA95D5
:10085000F1F71A95D1F6022FB22FBA95F1F70A9552
:10086000D9F73A9571F62898562C0895221B39E04D
:10087000001F3A9509F40895221F211B18F4210F37
:100880008894F6CF0894F4CF622C722CB0E0889450
:10089000B395221F331FE0F7379527958894912E43
:1008A000802E020B130B10F4192D082D10F48894D0
:1008B00001C00894661C771CBA9571F7172D062D98
:1008C0000895322D11232AF43A9500951095031BB3
:1008D000130BF894029F712C002D129F912C802CE9
:1008E0007894780C172D921C292DB4E06B2E269548
:1008F000179507956A94D9F7332321F00095109541
:10090000031B130B089500914E010430A9F1B0911F
:100910002D01B15008F010C0B0910101B093030156
:1009200020921701209218012092190120921A0199
:1009300020921B016F7B20C060904E016064B091DB
:100940000101B093020108E317EC209113013091EB
:10095000140136952795B62DBA9541F03695279511
:10096000B62DBA95BA9511F0369527950E94440494
:100970000093170110931801089566FF1BC00091A2
:100980001701B09102010B1B10911801120928F4F4
:100990000038BFEF1B0740F009C00F37120508F4FD
:1009A00005C00FE710E002C000E81FEF00931C0134
:1009B00010931D01089566FF39C000911C01B0918C
:1009C00019010B0F10911D01B0911A011B1F20E09E
:1009D00030911D0133230AF42A95B0911B012B1F7E
:1009E0001AF4203F40F00AC02F3008F407C00FEF80
:1009F0001FEF2FE003C000E010E020EF3091030173
:100A0000B09132013B1718F4332331F009C0B09193
:100A10001D01BB235AF004C0B0911D01BB2332F469
:100A20000093190110931A0120931B01089566FF8A
:100A300030C020916D0100911C01000F10911D012B
:100A4000111F0E94610411232AF40038BFEF1B0715
:100A500040F009C00F37120508F405C00FE710E099
:100A600002C000E81FEF002352F0B0910201B01B5A
:100A70000B2F18F0013008F00AC001E008C0009503
:100A80000F5FB09102010B0F08F001C00FEF009350
:100A90001E01089566FF2EC020916E0100911A017B
:100AA00010911B010E94610411232AF40130BFEF51
:100AB0001B0740F009C00F3F120508F405C00FEFF7
:100AC00010E002C001E01FEF112352F0B0911E01AF
:100AD000B01B0B2F18F0013008F00AC000E008C06E
:100AE00000950F5FB0911E010B0F08F001C00FEFD2
:100AF0000093030108950FEF677FB72FB670F1F4ED
:100B00006860B0911401B83008F0677FB0911401AB
:100B1000A9F00FEF109114010E943604F894B091DF
:100B200010010B9F112D002D7894112309F00FEF68
:100B3000B09135010B1710F4009135010093340189
:100B400008950E94E80874FFB0E074FDB0E0B06C56
:100B5000B0937C00B0917A00B068B064B0937A0032
:100B60000E94E00374FFB0E074FDB0E0B06CB0939D
:100B70007C00B0917A00B068B064B0937A00B09114
:100B80007A00B6FDFCCF0091780010917900B09109
:100B90007A00BF77B0937A000E942E0927EE209347
:100BA000430130E030934401732E7694622E6694B4
:100BB000620E731E262D372D0217130778F08090D2
:100BC0004301B7EEB80DB093430180904401B0E00B
:100BD000B81DB0934401260D371DEECF8090430120
:100BE000909044011091440116950091430107959E
:100BF00016950795B0914301B00FB0934101B091A4
:100C00004401B11FB093420123E0169507952A9540
:100C1000E1F720914F012A9529F420924301209277
:100C200044010AC02A9521F0800E911E2A95E1F711
:100C30008092430190924401089520914F01B09118
:100C40007A00B6FDFACF0091780010917900B0914A
:100C50007A00BF77B0937A00B0914501B395B09315
:100C60004501B83060F120924501B0916C01BB2381
:100C700021F1112329F0B0914601BF3F61F009C075
:100C8000B09146010B1739F020F4BB2321F0BA953F
:100C900002C0B395E1F300913201B0934601B03048
:100CA00050F400ECB03038F400E8B03020F400E448
:100CB000B03008F400E0009332017F7E08952130C7
:100CC00099F00F3FB3E01B0778F4B09143010B1785
:100CD000B09144011B0740F4B0913201BB23A9F04D
:100CE000BA95B093320111C0B0913201BF3F69F0A3
:100CF000B395B0933201B0915401B33031F4B09157
:100D00003201BC5F10F4B093320100913201B09116
:100D10000301B01B10F400910301B09133010B17D4
:100D200050F000913301B0913301BF3F21F0B091F9
:100D30003301B0933201B0914E01B43009F406C0D2
:100D4000B09134010B1708F00B2F502EB0914501D4
:100D5000B73009F47061089502E3F894B09170011E
:100D60000B9F012D000C001F7894B09132010B17DE
:100D700010F0009132010093010100930301502E05
:100D800000933501089520921301B8E0B093140147
:100D900008952091200130912101F8940091840060
:100DA00010918500200F311F309389002093880017
:100DB0006160B2E0B6BB78942091110130911201CC
:100DC0000093110110931201021B130B20911301C8
:100DD00030911401622E732EB4E08B2EB2E09B2E64
:100DE000B0911401B43010F08A949A94B83010F095
:100DF0008A949A94769467948A94E1F7261937092D
:100E0000992021F0169507959A94E1F7200F311F4C
:100E1000209313013093140108F00895BFEFB093AD
:100E20001301B09314010895209122013091230100
:100E3000F8940091840010918500020F131F109305
:100E40008900009388006160B2E0B6BB7894089591
:100E500060FDFECF0E9414070895B0915E010091DD
:100E60000E01023808F0B395003A08F0B395B63099
:100E700008F0B5E09B2EBCE08B2EB0911401B3308E
:100E800030F48394839482FF02C083948394B230BD
:100E900030F48394839482FF02C08394839471FF1F
:100EA00003C0B3E09B2E822C10911401009113011A
:100EB00024E0169507952A95E1F70819120928F0FC
:100EC000B02FB250B12FB20910F402E010E0312F70
:100ED000202F712E602E76946794B92DB330E9F0EF
:100EE000B0FD05C0060D171D262D372D06C0000FBD
:100EF000111F0250120922E030E0B92DB33068F022
:100F000020932401309325010093200110932101A7
:100F1000609222017092230108950093240110939E
:100F200025012093200130932101609222017092CB
:100F30002301089560FDFECF20912201220F309100
:100F40002301331FB72FB67021F020911301309188
:100F50001401F8940091840010918500020F131F72
:100F600010938900009388006160B2E0B6BB78946A
:100F7000089560612092160120E004C06061209213
:100F8000160120E2B72FB67009F06F7E789460FDED
:100F900005C0B0911601BB2309F0089501E063FF7D
:100FA0000AC0B0911401B33008F002E0B09114010E
:100FB000B63008F003E071FF01C006E060FD06C036
:100FC000B0911601BB2311F0789408951AE083FFC5
:100FD0001AE0789400000000F89462FD03C014E168
:100FE00083FF14E171FF01C018E7B091B2003091A6
:100FF0003901B31BB10B10F3B0911601B395B09347
:101000001601B5E03B2F6B2E722CB0B7B072B21741
:1010100009F073943A95C9F773947614A8F464FFB1
:10102000B1CF6F7E30918400609085007090130185
:1010300080901401370D681C6092890030938800FD
:101040006160B2E0B6BB9ECF64FD9CCF0A9509F00B
:10105000B5CF7894089571FF0AC0B0910D01B39592
:10106000B0930D0160FD0CC020920D0109C060FD20
:1010700007C064FD05C067FD03C0BF91BF911EC5D9
:1010800008952091240130912501F8940091840065
:1010900010918500020F131F1093890000938800A0
:1010A0006160B2E0B6BB789408950E94410800E008
:1010B00063FF03C064FF01C001E0F89410910E01CA
:1010C000B7E01B9F212D102D7894200F26951795A2
:1010D000269517952695179510930E01183718F435
:1010E000B8E7B0930E0100910E01B0910F010B17FC
:1010F00020F060622B982C982D9860FDFECF08950B
:10110000F8942A982898299882FF07C0EFE1F1E027
:1011100073FF03C0B1E4BA95F1F795FF2A9A95FDE4
:10112000299AB2E0B093150189C0F89495FF2D98E3
:1011300095FD2B9882FF0DC0EFE0F1E073FF0BC02F
:10114000289895FF299895FD2A98B1E4BA95F1F76A
:1011500002C0E9ECF0E062FF03C0552009F02C9AD0
:10116000B3E0B09315016AC0F8942A98289829989A
:1011700082FF07C0EFEFF0E073FF03C0B1E4BA9560
:10118000F1F795FF299A95FD2A9AB4E0B0931501DD
:1011900055C0F8942C9882FF0DC0EFEEF0E073FF7D
:1011A0000BC095FF2A9895FD29982898B1E4BA9527
:1011B000F1F702C0E1ECF0E062FF06C0552021F03B
:1011C00095FF2B9A95FD2D9AB5E0B093150136C089
:1011D000F8942A982898299882FF07C0ECEDF0E04F
:1011E00073FF03C0B1E4BA95F1F7289AB6E0B09363
:1011F000150124C0F89495FF2B9895FD2D9882FF3A
:1012000010C0E2E3F1E073FF0EC095FF2A9895FD50
:10121000299895FF299895FD2A98B1E4BA95F1F798
:1012200002C0E1EDF0E062FF06C0552021F095FF1D
:101230002D9A95FD2B9AB1E0B093150167FF0BC075
:101240000E942E09B1E4BA95F1F7B1E0BA95F1F731
:101250002A9A289A299A6F7D7894089520EC30E094
:10126000F9012B982C982D982A98289829986B7F0B
:101270000895ACE4B1E009E00D9309E00D9304E0BA
:101280000D9301E00D9303E00D930FEF0D930BE031
:101290000D9301E00D9301E00D9301E00D93A8E59E
:1012A000B1E001E00D930FEF0D930D930FEF0D9350
:1012B0000D930D9303E00D9306E00D930FEF0D9347
:1012C0000D9305E20D9300ED0D9308E20D9300E5FB
:1012D0000D9304E00D930DE00D9302E00D9300E0FB
:1012E0000D930AE70D930FEF0D9301E00D93089511
:1012F00020915F0109E011E0223011F405E011E0D6
:10130000233011F405E012E0243011F405E013E07D
:10131000253011F409E017E0263011F400E010E068
:1013200000933F0110934001209153018B7F777F01
:10133000B0915401B33019F09F7DB1FD90629F7B55
:10134000B0915501B1FD9064B22FB23011F08860B8
:1013500001C0877F0895E4E5F0E000914C010A9513
:10136000E00FF21DB491B0936D0100914D010A950B
:10137000E00FF21DB491B0936E010E942E09089502
:10138000E2E6F0E0009167010A95E00FF21DB491EA
:10139000B0936F010E942E090895E0E7F0E00091FC
:1013A00052010A95E00FF21DB491B09370010E94B2
:1013B0002E0908950895B09168010FEF1CE0B23036
:1013C00011F400EA1AE0B33011F402E815E00093DA
:1013D0000F0110931001089508952091620130913A
:1013E000630197FF02C020E03FEFB32FB21B6B2ECB
:1013F000B25810F4B2E86B2E00E00395609EB12D58
:10140000B058D8F3009347010895F894E3E0F0E072
:10141000B9E0B7BFB491B078C1F3F894A895B4B768
:10142000B070B4BFB0916000B861B0936000B0E03C
:10143000B0936000B4E0BEBFBFEFBDBF0E942E09F5
:10144000B0E0B5B9BFE3B4B9B0E0B8B9B0E0B7B98E
:10145000B0E0BBB9B0E0BAB92224A0E0B0E02D9270
:10146000AA31E9F7A0E0B1E00FEF2D920A95E9F774
:101470000E9439090E94820D0E9478090E94AB09DE
:101480000E94C0090E94CD090E94DA090E94DB096E
:101490000E94EC090E94ED0900916401009348014B
:1014A0000E942E09B2E0B5BDB2E0B0938100B2E077
:1014B000B093B100F8940E94EA030E94F5030E94E1
:1014C000E6030E94F8030E94E6030E94FB030E94C9
:1014D000E6030E94EA030E94EA030E94E803B1E0E7
:1014E000B5BBB0936E00B2E0B6BBB0936F00B1E095
:1014F000B7BBB0937000B0917B00B064B0937B0039
:10150000B0917A00B460B0937A000E94E0037894BE
:101510000E94A105B1E0BDBBBB27B160BCBB8D7F04
:101520000E94EA03B1E0B0930901626025E0B09146
:101530002C01BB2309F425E00E94E203B0912D01A8
:10154000B230A0F3B92FBF7100912F0100932E018B
:10155000B0932F01B01751F72A9549F76D7F96FF89
:10156000B3E096FDB2E0B0936900BB27B160BCBBAD
:101570008D7F0E94E8030E94E20302E0B92FBF7151
:1015800009F400E0B0912D01B017A8F3F8940E947F
:10159000F5030E94F5030E94F50378940E94EA0384
:1015A00020921F01B0915401B33009F48DC00E9404
:1015B000E203B0915801B13008F486C0B09109013E
:1015C000B13008F481C0B92FBF71F1F0B0912D0195
:1015D000BF3F08F479C0F8940E94FE0378940E94FB
:1015E000E803B0912D01B130B0F7F8940E94F503F3
:1015F0000E94E4030E94F50378940E94E803B091EE
:101600002D01BF3F90F378C3B3E09B2E9068F89410
:101610000E94ED0978940E94E803F8949F770E9455
:10162000ED0980902D01B0912D01BF37789408F419
:1016300053C00E94E003F8940E94FE0378949A94A9
:1016400029F7B82DB550B09363010E94EA03F894CE
:101650000E94B50D0E942D0E7894BAE09B2E9068E2
:10166000F8940E94ED0978940E94E803F8949F771B
:101670000E94ED0980902D01B0912D01BF37789423
:1016800060F70E94E003F8940E94F5030E94E403CF
:101690000E94F50378949A9411F7B82DBB5FB0932C
:1016A00062010E94EA03F8940E94B50D0E944A0E5E
:1016B00078940E94E803F8940E94ED097894B09120
:1016C0002D01BF3FB0F318C300912D01B0911F0150
:1016D0000B1710F000931F010E94E80301E0B09186
:1016E0005401B35009F405E0B0912D01B01708F092
:1016F00059CFF8940E94FE030E94FE030E94FE034D
:1017000078940E94EA032092090120920A01209213
:101710000B01B0910A01B395B0930A01BF3F79F56F
:10172000B0910B01B395B0930B01B091660109E143
:10173000BA9559F002E3BA9541F00DE7BA9529F050
:101740000AEFBA9511F020920B01B0910B01B0177E
:10175000B0F0B0910B01BA95B0930B01B4EBB0931C
:101760000A01B0916501B0934801F8940E94FE030C
:101770007894B0916401B09348010E94E8030E94FC
:10178000E403B0910601BB2321F4B92FBF7109F422
:10179000CCCEB0912D01B63008F4BBCFB09154013E
:1017A000B35011F00E94E803B0910601BB2309F485
:1017B000BCCEF8940E942E092092010120920201D1
:1017C00020920301522C7894B0915101B0933601CC
:1017D00020921701209218012092190120921A01DB
:1017E00020921B012092450160E070E020920E01E2
:1017F0000E94C306B8E0B093450170610E94E00307
:1018000074FFB0E074FDB0E0B06CB0937C00B091B8
:101810007A00B068B064B0937A00B0917A00B6FDF7
:10182000FCCF0091780010917900B0917A00BF77D9
:10183000B0937A00112309F00FEF009346010E9444
:101840001D06B8E0B0934501706180905301B2E08D
:10185000B09353010E94780980925301F894BFEF2E
:10186000B09332010E94AC06B0910101B0933201F5
:10187000B0933301B09334017894B1E0B093010197
:10188000B09303015B2EB0933B01B0913101B09353
:101890003A017160726020920D010E94E8080E9476
:1018A000FA080E94C9060E94C3060E942D0705C0BF
:1018B0000E947809209245017F7E95FFB5E095FD55
:1018C000B3E0B06CB0937C000E94BE070E942B086E
:1018D0000E9441080E9483040E9455080E948008CB
:1018E0000E94C9060E9428070E942D070E949A079D
:1018F000B4E0B06CB0937C000E94B9070E942B0842
:101900000E9441080E94BD040E947B050E94550868
:101910000E9495080E94C9060E9428070E942D0770
:101920000E949A0795FFB3E095FDB5E0B06CB093C7
:101930007C000E94BE070E942B080E9441080E9462
:10194000DB040E9455080E94B4080E94C9060E9448
:1019500028070E942D070E949A0795FFB5E095FD84
:10196000B3E0B06CB0937C000E94B9070E942B08D2
:101970000E9441080E9417050E9455080E94C9084C
:101980000E94C9060E9428070E942D070E949A07FC
:10199000B4E0B06CB0937C000E94BE070E942B089C
:1019A0000E9441080E944A050E9455080E94E808CA
:1019B0000E94C9060E9428070E942D070E949A07CC
:1019C00095FFB3E095FDB5E0B06CB0937C000E944C
:1019D000B90774FFB0E074FDB0E0B06CB0937C0068
:1019E000B0917A00B068B064B0937A000E942B087E
:1019F0000E9441080E9455080E94FA080E94C906E8
:101A00000E9428070E942D070E941D060E949A0727
:101A100071FF2EC067FD2CC0B0913501B09332012B
:101A2000B0933301B0913101B0933A01B1E0B0937A
:101A30003B0114E624E1B0910D01B11798F07D7FD0
:101A4000746020930C01B0915401B33051F4B09103
:101A50003501B0933201BFEFB0933301B0E2B093E0
:101A6000340106C0B0912D01B13008F026CF26C058
:101A700072FF10C067FD0EC0B0910C01BA9511F451
:101A80007B7F16CFB0930C01B0912D01B13008F0DF
:101A900014CF14C0B0913001BA3F80F4B92FBF7198
:101AA00021F4B0910601BB2349F0B091140100EF7D
:101AB00067FF01C000E6B01708F4FFCEF8940E945B
:101AC0002E0980905301B2E0B09353010E9478092F
:101AD0008092530120920101209202012092030181
:101AE000522C209236017E7F78940E94E0030E945F
:101AF0002E09B92FBF7129F4B0910601BB2309F457
:101B000014CD03CEEDE0F0E00E94AE0D053509F0F6
:101B10001EC0EEE0F0E00E94AE0D0A3A09F017C0D8
:101B20003AE0ACE4B1E0E3E0F0E00E94AE0D0D93EA
:101B300031963A95D1F735E1A8E5B1E0EFE0F0E074
:101B40000E94AE0D0D9331963A95D1F704C00E94D4
:101B500039090E94B50DE4E2F0E00895F999FECF4D
:101B6000E1BDF2BDF89A00B508950E94D80D3AE0A3
:101B7000ACE4B1E0E3E0F0E00D910E94D00D3196CD
:101B80003A95D1F735E1A8E5B1E0EFE0F0E00D914D
:101B90000E94D00D31963A95D1F70E94E30D089539
:101BA000F999FECF00BDE1BDF2BDFA9AF99A089508
:101BB000EDE0F0E00FEF0E94D00DEEE0F0E00FEF6F
:101BC0000E94D00D0895EDE0F0E005E50E94D00DF3
:101BD000EEE0F0E00AEA0E94D00D0895309149014C
:101BE00000914A01313011F400934C01323011F46C
:101BF00000934D01333011F400934E01343011F451
:101C000000935001353011F400934F01363011F438
:101C100000935201373011F400935E01383011F413
:101C200000936701393011F400935F013A3011F4E9
:101C3000009353013B3011F4009368013C3011F4E0
:101C4000009354013D3011F400935501089525E0AF
:101C50000E94EA032A95E1F708950E94F5030E9485
:101C6000F8030E94FB030E94FE030E94E4030E940B
:101C7000F5030E94F8030E94FB030E94FE030E94EA
:101C8000E4030E94F5030E94F8030E94FB030E94F4
:101C9000FE0308950E94FE030E94FB030E94F803C6
:101CA0000E94F5030E94E4030E94FE030E94FB03CE
:101CB0000E94F8030E94F5030E94E4030E94FE03C1
:101CC0000E94FB030E94F8030E94F5030895809090
:101CD000490190904A010E94F5030E94F5030E9479
:101CE000F5030E94E4038A94B1F70E94FE030E9468
:101CF000E4039A94D1F70895F8940E942D0E7894F5
:101D00000E94270E0E94270EB1E0B0934901B1E076
:101D1000B0934A0120924B01F8940E94670E789488
:101D2000B5E06B2E70902D010E94EA03B0912D0159
:101D30007B16C1F7B13018F0BF3F70F10CC00E94A4
:101D4000EE0DF8940E94B50D0E942D0EB8E0B093F0
:101D500060000E94270E6A9429F7B0914B01B39559
:101D6000B0934B01B33008F4D7CF0E94270EB09147
:101D70004A01B395B0934A01F894B0914901BA95DC
:101D8000EEE7F0E0EB0FF21D049178940395B0912B
:101D90004A01B01708F4BECF0E94270E0E94270EFA
:101DA000B0914901B395B0934901B0914901BE305A
:101DB00008F4ADCF0E943909F8940E94B50DB8E03F
:081DC000B09360000E94270EA1
:00000001FF
